:1000000038C053C052C051C050C05DC052C04DC076
:100010004CC04BC04AC049C048C047C046C045C09C
:1000200044C043C042C00829573F9F2D49CBA5314A
:100030000F76C73493F27E37D00D013AB60B613D8F
:100040002AAAAB3F0000003F80000000083B3BD7DE
:100050004ABC846E023D2FC1FEBD9A31743DDA3D2B
:1000600083BE117FC73E4CBBE5BEAAAA6C3F800091
:10007000000011241FBECFE5D2E0DEBFCDBF11E0EE
:10008000A0E6B0E0E2EEFEE103C0C89531960D9225
:10009000A635B107D1F711E0A6E5B1E001C01D9288
:1000A000AB3EB107E1F7E9D91BCFAACFC39AC398FA
:1000B00008951F920F920FB60F9211240F900FBE4A
:1000C0000F901F9018951F920F920FB60F92112448
:1000D0002F933F938F939F93EF93FF93909164019E
:1000E000E92FFF27EB5EFE4F80818DBD9F5F9093D0
:1000F00064012091E00188B38F7B822B88BB903410
:1001000059F4109264018091E5019091E601019605
:100110009093E6018093E50180916E01882309F5B3
:100120009091640180918D01981719F420642093B7
:10013000E00180916301981729F48091E0018F7BA1
:100140008093E0012091E5013091E60180916F01FB
:10015000909170012817390739F481E080936E017E
:1001600003C02F7B2093E001FF91EF919F918F912E
:100170003F912F910F900FBE0F901F90189582E81E
:1001800080BF81E08FBD89EF8BBD89B7846089BF57
:1001900008951092640110926E01F1DF7894089531
:1001A0008FEE8BBB8BBB86B39927847090700895BC
:1001B0008EEE8BBB8BBB86B39927847090700895AD
:1001C000C098B898C0980895B89AC0980895B89AF9
:1001D000C09A08951092E6011092E50110926E0106
:1001E0006091DB0177278AEF90E00CDE6F5F7F4F35
:1001F0007093700160936F0180916E018823E1F329
:10020000089510928D0180E280936301E3DF0895E9
:1002100080E280938D0110926301DCDF089580E11C
:1002200080938D0180E380936301D4DF089580E3A0
:1002300080938D0180E180936301CCDF0895EF927C
:10024000FF920F931F9313BE88B7836088BF14BAC1
:1002500012BE459B0CC08CEC85BB81E083BFB89A75
:10026000C09861E0E62EF12C012D112D0EC08CED11
:1002700085BB81E083BFB89AC09A5FEFE52E5FEF40
:10028000F52E5FEF052F5FEF152F88B79927837045
:100290009070892BD1F394DF63B322B308B601FECB
:1002A00003C081E080935701772788279927332758
:1002B000322F222744275527622B732B842B952B13
:1002C000512F402F3F2D2E2D82DD60938901709399
:1002D0008A0180938B0190938C011F910F91FF9065
:1002E000EF900895ACDF8DDFAADF609189017091F6
:1002F0008A0180918B0190918C014BDB6093E70127
:100300007093E8018093E9019093EA0181DF97DF20
:100310006091890170918A0180918B0190918C018B
:1003200038DB262F372F482F592F6091E701709126
:10033000E8018091E9019091EA0150DA20E030E093
:1003400040E05FE33BDC6093E7017093E80180935A
:10035000E9019093EA0163DF72DF60918901709196
:100360008A0180918B0190918C0113DB609379015C
:1003700070937A0180937B0190937C0158DF5FDF5B
:100380006091890170918A0180918B0190918C011B
:1003900000DB262F372F482F592F6091790170915C
:1003A0007A0180917B0190917C0118DA20E030E0A5
:1003B00040E05FEB03DC6093790170937A018093F6
:1003C0007B0190937C0108952F923F924F925F9210
:1003D0006F927F928F929F92AF92BF92CF92DF9255
:1003E000EF92FF920F931F93CF93DF93CDB7DEB7BA
:1003F00064970FB6F894DEBF0FBECDBF2091C30146
:100400003091C4014091C5015091C6012D873E87AE
:100410004F87588B80919F019091A001A091A101DD
:10042000B091A20189879A87AB87BC872091AB01E5
:100430003091AC014091AD015091AE012D833E83CE
:100440004F83588780919B0190919C01A0919D01C1
:10045000B0919E0189839A83AB83BC8329853A85B9
:100460004B855C856D857E858F859889B8D92D8172
:100470003E814F815885B3D929813A814B815C8176
:10048000AED92091AF013091B0014091B1015091AE
:10049000B201A5D920E030E040EA50E417DA698BD8
:1004A0007A8B8B8B9C8B609371017093720180931C
:1004B0007301909374012090DC013090DD01409035
:1004C000DE015090DF016090C7017090C8018090FC
:1004D000C9019090CA01A090BF01B090C001C09026
:1004E000C101D090C201E0907D01F0907E010091A9
:1004F0007F0110918001592D482D372D262D952DE6
:10050000842D732D622D6BD95D2D4C2D3B2D2A2D05
:1005100066D9512F402F3F2D2E2D61D920918E016C
:1005200030918F01409190015091910158D920E074
:1005300030E040EA50E4CAD96093BB017093BC013B
:100540008093BD019093BE0129813A814B815C81EA
:100550002093AF013093B0014093B1015093B201A9
:100560002D813E814F81588520939B0130939C01C2
:1005700040939D0150939E0129853A854B855C856A
:100580002093AB013093AC014093AD015093AE0189
:100590002D853E854F85588920939F013093A0017A
:1005A0004093A1015093A2012091790130917A01E9
:1005B00040917B0150917C012093C3013093C40191
:1005C0004093C5015093C601E0928E01F0928F01D5
:1005D0000093900110939101A0927D01B0927E0151
:1005E000C0927F01D09280016092BF017092C001E1
:1005F0008092C1019092C2012092C7013092C8013D
:100600004092C9015092CA012091E7013091E8015E
:100610004091E9015091EA012093DC013093DD0122
:100620004093DE015093DF016093E7017093E8018E
:100630008093E9019093EA0189899A89AB89BC8901
:100640008093790190937A01A0937B01B0937C0110
:1006500064960FB6F894DEBF0FBECDBFDF91CF9189
:100660001F910F91FF90EF90DF90CF90BF90AF90D0
:100670009F908F907F906F905F904F903F902F90C2
:10068000089510925A011092590180E090E001966D
:1006900090935A018093590125DE809159019091E0
:1006A0005A01853091059CF310925A01109259011C
:1006B00080E090E0A0E0B0E08093A3019093A401DB
:1006C000A093A501B093A60180935B0190935C0178
:1006D000A0935D01B0935E0180E090E0019690935D
:1006E0005A0180935901FEDD2091E7013091E80124
:1006F0004091E9015091EA016091A3017091A40138
:100700008091A5019091A6016AD86093A30170938E
:10071000A4018093A5019093A601209179013091C5
:100720007A0140917B0150917C0160915B01709155
:100730005C0180915D0190915E0151D860935B01F5
:1007400070935C0180935D0190935E0180915901EB
:1007500090915A018A3091050CF2089580915601CA
:100760008160809356018BBBC39AC3980895809192
:1007700056018E7F8260809356018BBBC39AC398CB
:100780000895809156018D7F809356018BBBC39A4B
:10079000C398089581E08093DB0110926D01089564
:1007A0008EEE8BBB8BBBB29908C090E08091580154
:1007B000882309F491E0909358018EEE8BBB8BBB9C
:1007C000B29BFBCF089580E690E074D75ADF08957E
:1007D00059D760E080E04CD782E690E06BD781E7A4
:1007E00090E068D70895DF92EF92FF920F931F93E6
:1007F000CF93DF93282F392FD62EEE24FF24F92F05
:10080000E82F81910894E11CF11C882321F080E1FC
:10081000E816F104B1F7D32FC22F00E010E0888171
:10082000882389F09F2D8E2D8D1991090197081726
:10083000190711F48EE22CD70F5F1F4F899128D72B
:100840000031110561F7DF91CF911F910F91FF905A
:10085000EF90DF9008956F927F928F929F92AF9268
:10086000BF92CF92DF92EF92FF920F931F9310925D
:10087000570138DD07D780915701882309F0B1C1AE
:100880006091E7017091E8018091E9019091EA019E
:100890003CDAE62EF72E082F192F6091790170911E
:1008A0007A0180917B0190917C012FDA262F372FDE
:1008B000482F592F912F802F7F2D6E2D90D7DFD964
:1008C00020E030E046EA55E481D888232CF481E02A
:1008D0008093DB0110926D0177DD6091650170916D
:1008E0006601809167019091680153D8262F372FB8
:1008F000482F592F6091E7017091E8018091E9013B
:100900009091EA016BD7662E772E882E992E6093F0
:10091000E7017093E8018093E9019093EA01609107
:10092000920170919301809194019091950131D839
:10093000262F372F482F592F6091790170917A0116
:1009400080917B0190917C0149D7A62EB72EC82EAD
:10095000D92E6093790170937A0180937B019093F3
:100960007C01992D882D772D662DCFD9E62EF72E77
:10097000082F192F9D2D8C2D7B2D6A2DC6D9262F42
:10098000372F482F592F912F802F7F2D6E2D27D74E
:1009900076D920915F0130916001409161015091C1
:1009A000620194D76093750170937601809377010B
:1009B00090937801592D482D372D262D9D2D8C2D66
:1009C0007B2D6A2D4ED7209181013091820140917B
:1009D00083015091840102D760939701709398012D
:1009E0008093990190939A0182E890E063D620E089
:1009F00030E040E251E460917501709176018091A0
:100A0000770190917801DAD8A7D72AE030E04BEC53
:100A100051E09DD661E080916D01681B8BEC91E007
:100A2000E2DE60E087E024D685E890E043D620E06F
:100A300030E143EB55E4609197017091980180910A
:100A4000990190919A01BAD887D72AE030E04BEC0F
:100A500051E07DD662E08BEC91E0C5DEA09075019F
:100A6000B0907601C0907701D0907801E090970126
:100A7000F09098010091990110919A01912F802F87
:100A80007F2D6E2D1DD7262F372F482F592F9D2DA7
:100A90008C2D7B2D6A2D92D86093B7017093B8018D
:100AA0008093B9019093BA01912F802F7F2D6E2DE5
:100AB000D3D8262F372F482F592F9D2D8C2D7B2DA6
:100AC0006A2D7CD86093E1017093E2018093E30189
:100AD0009093E40188E890E0EDD580915801882357
:100AE00009F58AE890E0E6D520E030E04AE754E4F2
:100AF0006091B7017091B8018091B9019091BA01EC
:100B00005DD82AD72AE030E04BEC51E020D663E0F4
:100B100080916D01681B8BEC91E065DE8DE890E0C3
:100B2000C9D523C08FE890E0C5D520E030E040E291
:100B300051E46091E1017091E2018091E3019091B3
:100B4000E4013CD82091B7013091B8014091B9013E
:100B50005091BA01BBD600D72AE030E04BEC51E00F
:100B6000F6D562E08BEC91E03EDE61E087E080D577
:100B700020E030E040E05FE36091E1017091E2014C
:100B80008091E3019091E40124D7181624F080911C
:100B9000DB01813079F182E990E08CD520E03EE6FE
:100BA00045E757E46091E1017091E2018091E30132
:100BB0009091E4018BD620E034E244E759E4FED77B
:100BC000CBD62AE030E04BEC51E0C1D562E0809119
:100BD0006D01681B8BEC91E006DE85E990E06AD53B
:100BE00009C088E990E066D58AE08093DB0181E066
:100BF00080936D011F910F91FF90EF90DF90CF9048
:100C0000BF90AF909F908F907F906F9008956F925C
:100C10007F928F929F92AF92BF92CF92DF92EF928C
:100C2000FF920F931F93CF93DF93CDB7DEB7249737
:100C30000FB6F894DEBF0FBECDBF90DD74E0F72E87
:100C4000A0E0B0E00C2F1D2F0F5F1F4FF12FE02F02
:100C50001F2C01D969817A818B819C817DD660931B
:100C60006501709366018093670190936801A4E029
:100C7000B0E0F12FE02F1F2CEED889819A81AB8153
:100C8000BC818093A7019093A801A093A901B09380
:100C9000AA01A8E0B0E0F12FE02F1F2CDCD8898159
:100CA0009A81AB81BC818093850190938601A0934A
:100CB0008701B0938801ACE0B0E0F12FE02F1F2C4A
:100CC000CAD889819A81AB81BC8180936901909354
:100CD0006A01A0936B01B0936C01D4D481EA90E0D7
:100CE000E9D420E030E040E251E460918501709168
:100CF0008601809187019091880160D72DD62AE0E6
:100D000030E04BEC51E023D560E08BEC91E06BDD03
:100D100085EA90E0CFD420E030E04AE754E46091E7
:100D2000690170916A0180916B0190916C0146D7C5
:100D300013D62AE030E04BEC51E009D562E08BECB1
:100D400091E051DD88E890E0B5D48AEA90E0B2D431
:100D50003ADD6091590170915A01882777FD80959D
:100D6000982F17D6E62EF72E082F192F262F372F5C
:100D7000482F592F6091A3017091A4018091A50182
:100D80009091A601A3D5E8D504D6262F372F482F5A
:100D9000592F6091B3017091B4018091B501909188
:100DA000B6011CD5D9D56093650170936601809317
:100DB000670190936801512F402F3F2D2E2D609198
:100DC0005B0170915C0180915D0190915E017ED527
:100DD000C3D5DFD5262F372F482F592F6091A70174
:100DE0007091A8018091A9019091AA01F7D4B4D57E
:100DF0006093920170939301809394019093950175
:100E0000B6DCE1DC8FEE8BBB8BBBB29BFCCF609181
:100E1000590170915A01882777FD8095982FB9D58F
:100E2000A62EB72EC82ED92E262F372F482F592F52
:100E30006091A3017091A4018091A5019091A601F8
:100E400045D5E62EF72E082F192F60916501709178
:100E5000660180916701909168019BD5262F372FFD
:100E6000482F592F912F802F7F2D6E2DB7D4662EAE
:100E7000772E882E992E5D2D4C2D3B2D2A2D60919D
:100E80005B0170915C0180915D0190915E011ED5C6
:100E9000E62EF72E082F192F609192017091930181
:100EA000809194019091950174D5262F372F482F6A
:100EB000592F912F802F7F2D6E2D90D4A62EB72ED7
:100EC000C82ED92E992D882D772D662D1ED7E62E6A
:100ED000F72E082F192F9D2D8C2D7B2D6A2D15D7C0
:100EE000262F372F482F592F912F802F7F2D6E2D92
:100EF00076D4C5D6E62EF72E082F192F60937501EC
:100F0000709376018093770190937801592D482D45
:100F1000372D262D9D2D8C2D7B2D6A2DA2D4209131
:100F2000690130916A0140916B0150916C0156D476
:100F30006093810170938201809383019093840177
:100F400020E030E040E251E4912F802F7F2D6E2D84
:100F500035D62091850130918601409187015091CD
:100F60008801B4D460935F01709360018093610144
:100F70009093620106DC84E0E1E8F1E0A0E1B0E0FA
:100F8000182E6ED7EFE5F1E0A4E1B0E0182E68D797
:100F9000E5E6F1E0A8E1B0E0182E62D7E2E9F1E081
:100FA000ACE1B0E0182E5CD724960FB6F894DEBF03
:100FB0000FBECDBFDF91CF911F910F91FF90EF90AA
:100FC000DF90CF90BF90AF909F908F907F906F9069
:100FD00008958FEE8BBB8BBBB29912C081E08093DA
:100FE000DB0110926D014ED38FEE8BBB8BBBB29B9E
:100FF000FCCFEEDB8FEE8BBB8BBBB299FCCF07DE59
:1010000008956F927F928F929F92AF92BF92CF92EC
:10101000DF92EF92FF920F931F938FEE8BBB8BBBF0
:10102000B29909C281E08093DB0110926D012AD34D
:101030008FEA90E03FD381E790E03CD38FEE8BBB0B
:101040008BBBB29BFCCF8FEE8BBB8BBBB299FCCF23
:1010500019D382EC90E02ED38AEC90E02BD3B3DB53
:101060006091590170915A01882777FD8095982FDA
:1010700090D4E62EF72E082F192F262F372F482F22
:10108000592F6091A3017091A4018091A5019091C5
:10109000A6011CD461D460936501709366018093AE
:1010A000670190936801512F402F3F2D2E2D6091A5
:1010B0005B0170915C0180915D0190915E0106D4AD
:1010C0004BD4609392017093930180939401909319
:1010D00095018FEE8BBB8BBBB29BFCCFD3D260E074
:1010E00080E0C6D287ED90E0E5D281E790E0E2D2E1
:1010F0008FEE8BBB8BBBB299FCCFC4D28BEE90E052
:10110000D9D28AEC90E0D6D25EDB8FEE8BBB8BBB64
:10111000B29BFCCF6091590170915A01882777FDED
:101120008095982F36D4A62EB72EC82ED92E262FCE
:10113000372F482F592F6091A3017091A4018091FE
:10114000A5019091A601C2D3E62EF72E082F192FE4
:1011500060916501709166018091670190916801CD
:1011600018D4262F372F482F592F912F802F7F2DBE
:101170006E2D34D3662E772E882E992E5D2D4C2D14
:101180003B2D2A2D60915B0170915C0180915D0186
:1011900090915E019BD3E62EF72E082F192F6091B8
:1011A0009201709193018091940190919501F1D3F6
:1011B000262F372F482F592F912F802F7F2D6E2DBF
:1011C0000DD3A62EB72EC82ED92E992D882D772D6A
:1011D000662D9BD5E62EF72E082F192F9D2D8C2DD1
:1011E0007B2D6A2D92D5262F372F482F592F912FDF
:1011F000802F7F2D6E2DF3D242D520E030E846E9D6
:1012000053E464D360935F01709360018093610144
:1012100090936201592D482D372D262D9D2D8C2D13
:101220007B2D6A2D1ED36093810170938201809380
:101230008301909384018FEE8BBB8BBBB29BFCCF61
:10124000C7DA8FEE8BBB8BBBB299FCCF1BD288EF7A
:1012500090E030D283DAB7DA6091590170915A0187
:10126000882777FD8095982F94D3E62EF72E082FA8
:10127000192F262F372F482F592F6091A3017091D6
:10128000A4018091A5019091A60120D365D381D3BB
:101290006093B3017093B4018093B5019093B6014C
:1012A000512F402F3F2D2E2D60915B0170915C01DD
:1012B00080915D0190915E0109D34ED36AD3609312
:1012C000A7017093A8018093A9019093AA014FDA16
:1012D0007ADA8FEE8BBB8BBBB29BFCCF609159014E
:1012E00070915A01882777FD8095982F52D3E62E6A
:1012F000F72E082F192F262F372F482F592F60919F
:10130000A3017091A4018091A5019091A601DED264
:101310002091B3013091B4014091B5015091B601D3
:101320005DD2662E772E882E992E512F402F3F2D7D
:101330002E2D60915B0170915C0180915D01909117
:101340005E01C4D2A62EB72EC82ED92E992D882D77
:10135000772D662DDAD4E62EF72E082F192F6091FF
:10136000920170919301809194019091950111D314
:10137000262F372F482F592F9D2D8C2D7B2D6A2DF1
:101380002DD2C3D4262F372F482F592F912F802F9E
:101390007F2D6E2D24D273D420915F013091600196
:1013A000409161015091620191D2609385017093E7
:1013B000860180938701909388012091A701309145
:1013C000A8014091A9015091AA019D2D8C2D7B2D42
:1013D0006A2D04D2592D482D372D262D42D2209129
:1013E0008101309182014091830150918401F6D1B5
:1013F0006093690170936A0180936B0190936C0113
:10140000C0D984E0E3EBF1E0A0E0B0E0182E28D5ED
:10141000E7EAF1E0A4E0B0E0182E22D5E5E8F1E03B
:10142000A8E0B0E0182E1CD5E9E6F1E0ACE0B0E0B1
:10143000182E16D5ECDB1F910F91FF90EF90DF90E7
:10144000CF90BF90AF909F908F907F906F900895B6
:101450001BBA8FE78ABB85E088BB8BE487BB80E43F
:1014600088B986B5806286BD8CE040D10BD11092E0
:1014700056011BBAC39AC3980895CF93DF93CDB793
:10148000DEB728970FB6F894DEBF0FBECDBF10921F
:10149000580180E090E0A0E0B0E08093810190935B
:1014A0008201A0938301B093840110926501109290
:1014B00066011092670110926801109292011092D9
:1014C0009301109294011092950180E090E4A3EFB3
:1014D000B4E480935F0190936001A0936101B093A5
:1014E000620180E090E0A4EEB1E4809385019093E6
:1014F0008601A0938701B093880181E08093DB018E
:1015000010926D01A5DF45D6BDD089E091E0D2D023
:10151000E9D6B8D076DD24E04C2F5D2F4B5F5F4FCE
:10152000A0E1B0E0F52FE42F122E95D48D819E819D
:10153000AF81B8858093810190938201A09383014C
:10154000B0938401A4E1B0E0F52FE42F122E83D4F0
:101550008D819E81AF81B88580935F0190936001FA
:10156000A0936101B0936201A8E1B0E04C2F5D2F20
:101570004F5F5F4FF52FE42F122E6DD489819A8132
:10158000AB81BC818093650190936601A093670154
:10159000B0936801ACE1B0E0F52FE42F122E5BD4DC
:1015A00089819A81AB81BC81809392019093930150
:1015B000A0939401B0939501F3D84DD94CD909DD8E
:1015C0004AD949D9F9CFDE9A00C0DE9808950F9321
:1015D0001F93082F662311F0DC9A01C0DC98DD9878
:1015E0008AB38F608ABB1BB3107F802F82958F7068
:1015F000812B8BBBE8DF0F70012B0BBBE4DF1F607F
:101600001BBB1F910F910895882311F0DC9A01C034
:10161000DC98DD9A8AB3807F8ABBDE9A00C089B3EA
:10162000DE9800C0DE9A00C099B3DE988295807F74
:101630009F70892B9927089580E0E6DF87FDFCCF16
:1016400082E090E00197F1F780E0DEDF99270895CE
:101650001F93182FF1DF60E0812FB9DF1F910895EC
:101660001F93182FE9DF61E0812FB1DF1F910895EB
:10167000662311F4805801C08054EADF0895DCDF4E
:101680009927089581E0E4DF089582E0E1DF08957D
:101690001F93182FD1DF1A3041F4803410F480E406
:1016A00001C080E08058D4DF03C061E0812F8FDF6C
:1016B0001F910895CF93DF93D92FC82F01C0E8DF82
:1016C00089918823E1F7DF91CF910895CF93DF933C
:1016D000D92FC82F01C0DCDFFD2FEC2F2196C89534
:1016E000802D8823C1F7DF91CF910895FF920F934A
:1016F0001F93F82E8AB38F678ABB80E89EE3019719
:10170000F1F7D99AD89A5FDF80E893E10197F1F772
:101710005ADF00E410E0912F802F0197F1F753DF9B
:10172000912F802F0197F1F7D8984DDF912F802FBF
:101730000197F1F788E28CDF88E08ADFA3DF86E09B
:1017400087DF8F2D85DF1F910F91FF900895E42F84
:10175000F52FCF93FF93EF9322304CF125323CF5D8
:10176000C22FE894CA3049F497FB3EF490958095D7
:10177000709561957F4F8F4F9F4F2C2F33274427B4
:101780005527FF93EF9385D3EF91FF91605D6A3307
:101790000CF0695D6193622F732F842F952F605039
:1017A00070408040904049F716F4CDE2C19310821A
:1017B0008F919F91CF9100C0A82FB92FE82FF92FBB
:1017C000672F71917723E1F7329704C07C916D9375
:1017D00070836291AE17BF07C8F308955058192E51
:1017E0008FD101D038C1BA176207730784079507F4
:1017F000B1F188F40EF410940B2EBA2FA02D062E02
:10180000622F202D072E732F302D082E842F402D70
:10181000092E952F502DFF275523B9F0591B49F05C
:10182000573E98F0469537952795A795F0405395E4
:10183000C9F776F0BA0F621F731F841F30F48795C3
:1018400077956795B795F040939517FA0F2E089501
:10185000BF1BBB27BA0B620B730B840BF6CFDEF6F4
:101860007BC1552319F0992351F017C09923A1F09A
:1018700097FB6BED7FE089EC9FE397F90895552383
:1018800059F02AF46BED7FE089E490E4089566272F
:101890007727882799270895F6C01F93112797FD6A
:1018A000116057FD126012D035D211FF07C02BED29
:1018B0003FE049E450E410FD506891DF1F91089526
:1018C00050E449EC3FE02BED6ED0A2C019D101D01D
:1018D000C2C0552359F0992369F09F575F57951B54
:1018E00033F442F4903811F4915805C0CCC09158AB
:1018F0009F3F09F431C1BB27112462177307840786
:1019000030F4660F771F881FBB1F915098F311D0DA
:101910000F920FD00F920DD0A0E826173707480777
:101920001B0609F0A048BA2F602D7F918F910024EB
:101930000895A0E80024621773078407B10528F012
:10194000621B730B840BB1090A2A660F771F881F6D
:10195000BB1FA69581F7089597FBDED09F3738F01F
:10196000FEE9F91B982F872F762F6B2F05C0F1C04A
:101970009695879577956795F150D0F73EF49095B9
:101980008095709561957F4F8F4F9F4F0895E89494
:1019900003C097FB0EF4F3DFB62F672F782F892F44
:1019A0009EE9002458C05F77552319F444230AF0B8
:1019B0006AC02F933F934F935F9388DF5527442747
:1019C000CDD05F914F913F912F91F8C00ED05EF036
:1019D00004C00BD026F001C008D019F020F48FEF1E
:1019E000089580E0089581E0089597FB092E05266B
:1019F00000F8689488D0E89407FC07C06217730762
:101A00008407950721F008F40094079498940895AA
:101A10001F939F7750EC49E43FE02BEDE0DE10E8A8
:101A20009F775FE349EC3FE02BED62177307840774
:101A3000950720F050EC49E4D2DE112766D190687A
:101A4000E6E2F0E023D091271F9108959A95BB0F0D
:101A5000661F771F881F11249923A1F08823B2F7EE
:101A60009F3F59F0BB0F48F421F4002011F460FFB0
:101A700004C06F5F7F4F8F4F9F4F881F979587954B
:101A800097F9089566C09FEF80EC0895FF92EF925A
:101A9000DF92CF92BF92C62ED72EE82EF92EC89590
:101AA000B02C319619D0C895B02C3196BB2071F06E
:101AB0009F938F937F936F936C2D7D2D8E2D9F2DF4
:101AC0000BD02F913F914F915F9100DFBF90CF904E
:101AD000DF90EF90FF90089548D104C02C2D3D2D4C
:101AE0004E2D5F2DEF93FF9369D0FF91EF913DD184
:101AF000EF93FF9374DEFF91EF91BA9479F7089515
:101B0000052E092607FA440F551F5F3F79F0AA27D3
:101B1000A51708F051E04795880F991F9F3F31F0B6
:101B2000BB27B91708F091E0879508959F919F9181
:101B30001124A9CF97FB880F991F9F3F31F0BB2736
:101B4000B91708F091E0879508959F919F9111240E
:101B50009ACF66277727882799270895EBDFCF93B9
:101B6000DF93D52FC42F55274427332722279923C6
:101B7000D9F09F37C8F0F92F6EDF592F482F372F34
:101B8000262FF63968F4E8DE04DFC030CD0721F0F7
:101B900069937993899399939058DF91CF911FCE50
:101BA0009927882777276627C030CD0721F029930A
:101BB000399349935993DF91CF914DCFA1DF01D054
:101BC0004ACF992339F0552329F09F575F57950F36
:101BD00013F4CAF1C1CF91589F3FE1F3A62F00241F
:101BE0001124BB2766275527F8E0A69520F4020E9E
:101BF000131EB41F651F220F331F441F551FFA9574
:101C0000A1F7F8E0E72F7727F8E0E69520F4130E28
:101C1000B41F651F7A1F330F441F551FAA1FFA9563
:101C2000A1F7F82F8827F69520F4B40F651F7A1FC7
:101C30008E1F440F551FAA1FEE1FFF23A1F78823F5
:101C40001AF4939539F41FCF000C111CBB1F661FAB
:101C5000771F881F012808959F939F77993358F025
:101C600050E449EC3FE02BED9EDE5FEB49EC3FE0BA
:101C70002BEDB5DDCDDE5F9150789527089597FD6A
:101C800002CF992309F40895482F54DFF92FFF5705
:101C9000F5959F1B9F1BFF93DEDEFF92EF92DF9275
:101CA000CF92BF92AF929F928F92C62ED72EE82EE0
:101CB000F92E405847953327222740685FE36C2D63
:101CC0007D2D8E2D9F2D822E932EA42EB52EFEDDE2
:101CD000282D392D4A2D5B2D82DD4FEF5FEF5BD034
:101CE000262F372F482F592F82169306A406B506A4
:101CF00031F78F909F90AF90BF90CF90DF90EF9093
:101D0000FF905F9117DF950FA6CE262F372F482F14
:101D1000592F54CF1F930F930027192F10789F77B7
:101D20005FE340E8613071058407950710F00068B3
:101D300029D0912B6F937F938F939F93E6DFECE4F1
:101D4000F0E0A4DE5F914F913F912F9137DF0023A8
:101D500049F02BED3FE049EC5FE300E8902717FDE9
:101D600050683DDD0F911F910895C895502D319613
:101D7000C895402D3196C895302D3196C895202DA7
:101D800031960895262F372F482F592F9FE380E84B
:101D9000772766279BCDCEDE992359F0AA27940F8B
:101DA000A51F43F032F04FEF50E09417A50714F44D
:101DB00052CECFCE0EF006C000C09FEF80E870E09C
:101DC00060E008959FE780E870E060E00895FF27F5
:101DD000EE27BB27AA2760FF04C0A20FB31FE41F92
:101DE000F51F220F331F441F551F96958795779532
:101DF000679589F70097760771F79F2F8E2F7B2FB6
:101E00006A2F089597FB092E07260AD077FD04D084
:101E10000CD006D000201AF4709561957F4F08957C
:101E2000F6F7909581959F4F0895AA1BBB1B51E132
:101E300007C0AA1FBB1FA617B70710F0A61BB70B3A
:101E4000881F991F5A95A9F780959095682F792F2B
:101E50008A2F9B2F089509D001921A94E1F70895D3
:101E600001900BD01A94E1F70895E199FECFBFBB22
:101E7000AEBBE09A11960DB20895E199FECFBFBBBB
:101E8000AEBB0DBA11960FB6F894E29AE19A0FBE66
:101E90000895A1E21A2EAA1BBB1BEA2FFB2F0DC02F
:101EA000AA1FBB1FEE1FFF1FA217B307E407F5070A
:101EB00020F0A21BB30BE40BF50B661F771F881FE6
:101EC000991F1A9469F76095709580959095262FC3
:101ED000372F482F592F6A2F7B2F8E2F9F2F089532
:021EE000FFCF32
:101EE2002A0052656D6F7665206465766963650ABE
:101EF2000070726573732063616C20627574746F15
:101F02006E005A3D00413D000A00523D0020005142
:101F12003D004C3D006D48004F766572666C6F77F0
:101F2200005A3D200020413D20002063616C005397
:101F3200686F72742070696E732C207468656E20ED
:101F42000A0053686F72742E0A00506C65617365E3
:101F520020776169742E0033302E31204F686D2056
:101F62006F6E2070696E732C200A0052657369735C
:101F720074616E63652E0A004D6561732E20496E91
:101F8200742E205265662E0A00316B6C6D3038302B
:101F920038313342007C6F63574C41362D231B147A
:101FA2000E0804010000000104080E141B232D3644
:101FB200414C57636F7B8894A0ABB6C1CAD4DCE3B3
:101FC200E9EFF3F6F7F8F7F6F3EFE9E3DCD4CAC189
:061FD200B6ABA0948800EC
:00000001FF
